:100000007CC1B0C17FC494C193C1B1C491C190C13E
:10001000DEC48EC1D1C48CC18BC18AC189C1040325
:1000200009045A0368006100660074006D006100F5
:100030006E006E00230073006F006600740077008E
:1000400061007200650020002800770077007700CB
:100050002E00740075002D006300680065006D00BF
:100060006E00690074007A002E00640065002F00A5
:100070007E006800650068006100290026034600D4
:1000800075006E006B005500730062003A0050006E
:10009000720065006600650074006300680065001A
:1000A00072003A0368006500680061004000680063
:1000B00072007A002E00740075002D006300680045
:1000C00065006D006E00690074007A002E00640007
:1000D00065003A0030003000300038001201100195
:1000E00000000008C016D92700010102030109021F
:1000F0002200010100803209040000010300000019
:1001000009210101000122D7000705810308000A27
:1001100005010904A101850115002501750195015D
:1001200005090901810295078101C00600FF090147
:10013000A1018502150026FF007508950B0921B164
:10014000029501A48503193129359505B102751071
:10015000950226FF03350046001455046721D1F0AF
:100160000019362937B102B4A4850425017501951B
:10017000081940294781027510950126FF033500B3
:1001800046001455046721D1F0000B300084008133
:100190000216E60026720136E90046660155006740
:1001A000010001000B360084008102B4A4850525FE
:1001B0000A75049502092325FFB18275409514093B
:1001C00024B182751095320925B182B485060926BD
:1001D000B182751026DF010927B182752025FF96AF
:1001E000E0010928B182C0243337363534342F3347
:1001F000323130302B2F2E2D2C2C272B2A2928283A
:10020000372726252400544A4C495E46393B4B4D3E
:100210003C4E57385A485C52424450563F5D3E4728
:100220005B513D41007060656B636C716E69736119
:1002300062676A6468666F6D7200BBAB0A0E3D024E
:1002400022FC00C5740F736506DFE607F70E0D6D1F
:100250004F08909703E9110CA1D80B3859051C835E
:100260000984C2014ABA0456200E64C5028D1B09D6
:1002700028D2050B580DD1490CBA370E93010F52F5
:100280007D081C9306C5FA07A7E00BF02F01E9666D
:10029000007FB40A36AC044E8E03C1B70877CC0099
:1002A0003D430DB3FF0FAA5801E0660C0CEB036F42
:1002B000350614820B882A04F699092BDD05D20035
:1002C0000A9971075E140245AE0E1F4E0370B10D00
:1002D00096F700D3700CB318090B5206FCAA0FEE68
:1002E0009F0B81D501426B0ECACC08343D0AA50490
:1002F0000258830729E90467260511241FBECFE5AC
:10030000D2E0DEBFCDBF10E0A0E6B0E0EEE8F3E162
:1003100002C005900D92A436B107D9F711E0A4E60A
:10032000B0E001C01D92AE3DB107E1F74DD42DC83C
:1003300067CEA82FB92F80E090E041E050EA6095A9
:100340006F5F58F42D9138EF82279795879510F0BD
:10035000842795273F5FC8F3F3CF0895EADF8D9395
:100360009D930895CF93CFB7CF93C395B29BE9F7F1
:10037000B29B0EC0B29B0CC0B29B0AC0B29B08C01D
:10038000B29B06C0B29B04C0C2B7C8BD8D9ACEC096
:100390000F92DF93C0918200DD27C757DF4F012EF8
:1003A000B29B03C0DF910F90E3CF2F930F931F9366
:1003B0004F932FEF4F6F06B302FB20F95F933F93EC
:1003C00050E03BE065C016B30126502952FDC895A8
:1003D00056B3012702FB25F92F7306B3B1F050275E
:1003E000102712FB26F906B22230F0F000C016B337
:1003F000012702FB27F90126502906B22430E8F52F
:100400004F77206816B30000F6CF50274F7D20624B
:1004100006B2102F000000C006B300265029102796
:1004200012FB26F906B2E2CF4F7B06B3206400C070
:10043000DACF01265029167006B269F14E7F21608D
:10044000012F16B328C0002650294D7F06B2226026
:10045000102F29C0012650294B7F06B22460012F9E
:100460002DC016B301265029477F2860000006B230
:100470002EC04F7E06B3206130C0422706B3499399
:1004800000265029102706B24FEF12FB20F9297FD2
:1004900016B379F2167049F10126502906B20127E8
:1004A00002FB21F9237F06B371F200265029315057
:1004B000D0F006B2102712FB22F9277E16B351F2B4
:1004C00001265029012702FB06B223F92F7C49F2AD
:1004D000000006B3102712FB24F90026502906B2AB
:1004E0002F7939F270CF002717C03B503195C31BCD
:1004F000D0400881033CF1F00B34E1F02091800002
:100500001981110F1213EFCF4A81441F093639F1B7
:100510000D3211F0013E39F7009387003F915F9152
:100520004F911F910F912F91DF910F90CF91CFBFDE
:10053000CF91189500918700002381F310918500D9
:10054000112379F534307AF13093850000938100DE
:10055000109182003BE0311B3093820024C0009157
:1005600085000130F4F40AE54F7049F430916100E0
:1005700034FD1AC000936100CAE6D0E019C0309182
:10058000620034FD11C000936200C5E7D0E010C0E6
:10059000052710E000C021C0052710E0C89508BB62
:1005A00014C03AE501C032ED032EC0E0D0E032E0E5
:1005B00017B31660C29A08B317BB56E020E84FEF96
:1005C00020FF052708BB279517951C3F28F700003B
:1005D0004552B0F720FF0527279508BB17951C3F0C
:1005E000B8F629913A9561F7097F10918600110FAD
:1005F00008BBC250D04011F010938000046017B3C4
:10060000197F402F497F54E05A95F1F708BB17BB7B
:1006100048BB84CF8BB780648BBF8BE4809375001D
:1006200008951F93DC01162F8091620084FF0AC099
:100630008091750098E8892780937500912FE6E7EF
:10064000F0E007C08AE580936200F8CF8D91819336
:1006500091509923D9F786E790E0612F7FDE1C5FE8
:10066000109362001F9108950F931F93CF93DF9310
:100670006091850016160CF0D1C080918200CCE00C
:10068000D0E0C81BD109C757DF4F6350809181006C
:100690008D3209F0A6C08AE580936100683009F0C8
:1006A000B3C08881807609F08AC010927300898176
:1006B000882351F41092740083E790E090938400B3
:1006C0008093830032E085C0853021F48A81809355
:1006D00086000EC1863009F056C08B81813041F40E
:1006E0008CED90E0909384008093830032E103C10D
:1006F000823041F48EEE90E09093840080938300EA
:1007000032E2F9C0833051F58A81882341F48EE1C9
:1007100090E0909384008093830034E0ECC08130BB
:1007200041F482E290E090938400809383003AE564
:10073000E2C0823041F48CE790E090938400809393
:10074000830036E2D8C0833009F0D4C082EA90E05A
:1007500090938400809383003AE3CDC0813241F4CA
:1007600080E091E0909384008093830039E0C3C0DF
:10077000823209F0BFC080E191E0909384008093C1
:10078000830037EDB8C0883019F488E890E00AC0DB
:10079000893021F48A8180938800AAC08A3041F48C
:1007A00083E790E0909384008093830031E011C050
:1007B0008B3009F09DC08BE48093750099C0CE0109
:1007C0008AD1382F8F3F29F4888187FD3E81832F7E
:1007D00019C020E88F818823D1F48E818317C0F05F
:1007E00016C08091640087FD0FC0CE0153D28F3FA9
:1007F00021F48EE18093610004C0882311F080E031
:1008000001C08FEF20E004C080E020E801C0832F0A
:1008100020936400809360001092850080916100B5
:1008200084FF5BC0809160008F3F09F456C0182F91
:10083000893008F018E0811B80936000809164008B
:1008400080FD02C00BE401C003EC8F5F8093640065
:1008500087FF26C0209183003091840086FD05C06B
:10086000D901912FEBE6F0E011C0ABE6B0E080E0FB
:1008700090E006C0F901E80FF91FE491ED930196AD
:100880001817C1F705C08D91819391509923D9F71D
:10089000F901E10FF11DF0938400E093830009C09A
:1008A000112339F08BE690E0612F5DD2182F89304B
:1008B00060F48BE690E0612F51DD912F9C5F183042
:1008C00041F08FEF8093600004C08FEF8093600051
:1008D0009EE100936A00909361009AE086B386706F
:1008E00061F49150D9F7109286001092800005C0F3
:1008F00030E06FCF30E020EC6DCFDF91CF911F91D2
:100900000F9108951F920F920FB60F9211248F939B
:100910009F9380E48BBF7894889A899A8A9A06B4C8
:1009200003FE03C082B78093C3018091C3019091FD
:10093000C4019093BC018093BB01B39907C081E0CF
:100940008093BE018091C601816005C01092BE01F6
:100950008091C6018E7F8093C601F89480E68BBF9C
:100960009F918F910F900FBE0F901F9018957894C4
:100970001F920F920FB60F9211248F939F93809125
:10098000C3019091C40106B403FE03C080509F4F81
:1009900001C001969093C4018093C30183B390E09A
:1009A0008F739070892B09F48B9A9F918F910F9080
:1009B0000FBE0F901F90189578941F920F920FB64C
:1009C0000F9211240F900FBE0F901F9018957894DE
:1009D0001F920F920FB60F9211242F933F934F93B4
:1009E0005F936F937F938F939F93AF93BF93EF9397
:1009F000FF9387B190E0809590958F709070892BD0
:100A000059F484B195B19093CA018093C901899A30
:100A100016B88BE080BD23C03C9912C064B175B19B
:100A200080E090E02EE630E040E050E06AD4672FAE
:100A3000782F892F99277093C8016093C7010CC044
:100A400084B195B121E08039920710F43C9806C03A
:100A50009093C8018093C7018FE887B9369AFF91B8
:100A6000EF91BF91AF919F918F917F916F915F9126
:100A70004F913F912F910F900FBE0F901F9018959F
:100A80008091680090916900892B09F58F982091D9
:100A900066003091670081E02B3C380729F4F901AA
:100AA000359780818F708083235C314081F480E8AA
:100AB00098E1909367008093660080E897E09093B8
:100AC0006900809368008F9A21E030E002C020E046
:100AD00030E0C9010895FC0180818076803209F000
:100AE00071C08181813009F04AC082818330B9F1BF
:100AF000843030F4813069F0823009F063C011C075
:100B0000853009F448C0853090F1863009F05AC02C
:100B10004BC08DEB91E0909384008093830082E042
:100B2000089506B403FE03C082B78093C301809189
:100B3000C3019091C4019093BC018093BB012091AB
:100B40009F003091A000821B930B35E0969587950E
:100B50003A95E1F78093B20181EB91E002C087EA18
:100B600091E090938400809383008AE0089585EC5F
:100B700091E0909384008093830086E0089589300B
:100B800009F58281853039F0863071F08330D1F4F7
:100B900087EA91E002C081EA90E090936700809339
:100BA00066008681978108C08FEB91E09093670083
:100BB0008093660084E090E09093690080936800E1
:100BC0008FEF089580E0089594B714BE479A88E1A6
:100BD00081BD11BC11BA93FF0AC086B3867039F08B
:100BE00080E48BBF80E385BF78948895F89480E299
:100BF00085BF8BE080BD81E187BBC39A88B388BB8A
:100C0000C09AA59A18E015BB80E68BBF92E093BF0F
:100C100099BF81E08093BD019093B10183E08093FF
:100C2000A70184E08093C50185E08093A10086E060
:100C30008093BF01EFDC11BD78948895A8958D9BBA
:100C400013C098B59E5080916500981B88B580931D
:100C500065008D98993F1CF481B78F5F81BF9830F4
:100C60001CF081B7815081BFFFDC7CD18091620094
:100C700084FFE3CF889B06C08DEB91E062E0D1DC7E
:100C80008898DBCF899BD9CF85EC91E066E0C9DC01
:100C90008998D3CFDF92EF92FF920F931F93CF9358
:100CA000DF93EC01E62E40916800509169004115F8
:100CB000510509F44EC0EE2009F44BC0D42E8E2D00
:100CC00090E04817590710F4F42E01C0FE2C8F9BBA
:100CD00012C00F2D10E08091660090916700BE0158
:100CE000A80198D0809168009091690080179107C1
:100CF00051F4ADD008C08091660090916700BE01AC
:100D00004F2D50E039D30F2D10E080916600909167
:100D10006700800F911F9093670080936600809119
:100D2000680090916900801B910B909369008093FB
:100D30006800A6DE892B21F0C00FD11FED18B3CFBC
:100D400020E08091680090916900892B19F421E0DE
:100D500001C02FEF822FDF91CF911F910F91FF9054
:100D6000EF90DF900895DF92EF92FF920F931F9321
:100D7000CF93DF938C01E62E40916800509169007B
:100D800041155105E9F1EE20D9F1D42E8E2D90E0D8
:100D90004817590710F4F42E01C0FE2C8F9B09C090
:100DA0006091660070916700C8014F2D50E096D0A9
:100DB00008C06091660070916700C8014F2D50E037
:100DC000DBD2CF2DD0E080916600909167008C0F30
:100DD0009D1F9093670080936600809168009091BA
:100DE00069008C1B9D0B909369008093680048DE1E
:100DF000892B11F44F2D05C00C0F1D1FED18BCCF12
:100E00004FEF842FDF91CF911F910F91FF90EF90C3
:100E1000DF900895CF93DF93EC0141155105A1F0C8
:100E200020E030E0FE01E20FF31F81B3EF73F070BA
:100E3000E252FE4FDB01A20FB31F8C9180832F5F24
:100E40003F4F4217530771F7DF91CF9108958E9B63
:100E500021C020911E0230911F02E199FECFAEED1C
:100E6000B1E083E0F90180935700E895F90141E092
:100E70008D919D910C0140935700E8951124329675
:100E800082E0AE31B807A1F785E0F9018093570001
:100E9000E8958E980895DC01E1991CC04115510533
:100EA000C9F0FB01BFBBAEBBE09A8DB3908189173F
:100EB00039F09DBBF894E29AE19A78949F010CC0B6
:100EC0008EB39FB301969FBB8EBB4150504011F033
:100ED0003196EACF20E030E0C90108951F93CF9307
:100EE000DF93EC018E9B24C04115510511F18091D7
:100EF0001E0290911F029B01281B390BD901A2529F
:100F0000BE4F80E090E0FB01E80FF91F203431056F
:100F100010F41C9101C01491FE01E80FF91F108319
:100F200001962F5F3F4F11964817590761F701C08F
:100F30001AD2DF91CF911F91089506B403FC08C027
:100F4000F89480E886BD88E086BD82B382BF78943D
:100F5000089586B5F89480E886BD16BC82B782BB3A
:100F6000789408958B9B0CC08B988AE080BD80E9B3
:100F700087B906B403FC02C08FED01C088ED86B9C5
:100F80008A9B03C081B3847081BB0895DC011696EF
:100F90002C911697E22FFF27E7FDF095CF016DE624
:100FA00070E09DD13197F595E795F595E795582F28
:100FB0005E0F15968C911597682F772767FD7095B2
:100FC00041E030E02370307012C0423039F4211516
:100FD000310511F48DE109C08CE107C0842F86959D
:100FE0008695869584278170825E580F4F5F842F87
:100FF00090E0861797074CF313968C918D5B850FC5
:101000000895CF93DF93EC01C1DF282F9A819E5F73
:101010008F81981B983110F02F5F98512093C00159
:10102000892F90E064E170E05AD19C01898163E0EE
:1010300081D1992787FD9095820F931F9093C201CC
:101040008093C101DF91CF910895FC018281829547
:10105000880F807C918196959695892B80932402A8
:1010600082818695869586958F7080932502089556
:10107000FC018181880F880F880F807F9091250265
:10108000892B809325028181928125E09695879511
:101090002A95E1F780932602828182958695837056
:1010A0008093270284818F778093290285818F73B3
:1010B00080932A0286818F7380932B028781829589
:1010C000880F807E9085892B80932C028185809368
:1010D0002D020895FC018181880F8C7F9091270259
:1010E000892B8093270281819281880F892F881F05
:1010F000990B9195809328025BD0609320027093A6
:101100002102809322029093230297FD1BC083EB60
:1011100091E077DF8091C001809323028091C1012B
:101120009091C201880F991F880F991F8058974E80
:1011300060E272E044E050E06DDE8091C6018062C2
:101140008093C6010895503131F0583021F0573066
:1011500011F0533009F400D0B794A79494FAB7F87B
:101160009794879470FA93F8779408956627772771
:1011700011C0BA2FA695A695A69521E0B77019F0D3
:10118000220FBA95E9F70C900222B015661F771F5F
:10119000881F991FA591AA2361F708956594579414
:1011A0004794379420FA67F827948A95B9F70895F9
:1011B000E4E2F2E02F923F924F925F926F927F9221
:1011C0008F929F92AF92BF92CF92DF92EF92FF9257
:1011D000A2E0B0E05AE001900D925A95E1F750E19B
:1011E000B2DFE7EEF1E0C2DF6B017C01E6E0F2E0A6
:1011F000BDDFC626D726E826F9262FE03327442769
:10120000662777278827EC2DEF730E2E000C0E0E25
:10121000EAE3F2E0E00DF11D05900222602905905D
:1012200003227029C8950422802996E0F694E79459
:10123000D794C7949A95D1F794E0220F331F441F97
:101240009A95D9F7403FF9F66B017C01E5E2F2E0AF
:101250008DDF26263726482684E1A0DF5A9501F641
:1012600084E09CDF81E095E282199309B201862D2A
:1012700021F06FEF7FEFCB010894FF90EF90DF90AC
:10128000CF90BF90AF909F908F907F906F905F9026
:101290004F903F902F900895202FE4E2F2E0322FFC
:1012A000269526952695E20FF11D21E0377019F05D
:1012B000220F3A95E9F70080022600820895FC018A
:1012C000262FEDCF75DF50F40F930027E5DF70DF99
:1012D00020F4E2DF03950832C9F70F9108955527EE
:1012E000002480FF02C0060E571F660F771F61158E
:1012F000710521F096958795009799F7952F802D88
:101300000895FF27EE27BB27AA2760FF04C0A20F7E
:10131000B31FE41FF51F220F331F441F551F96955F
:1013200087957795679589F70097760771F7CF01CD
:10133000BD01089587FB082E062687FD819567FD70
:10134000619505D00EF4919507FC81950895991B40
:1013500079E004C0991F961708F0961B881F7A95AC
:10136000C9F780950895FB01DC0102C005900D923C
:1013700041505040D8F70895FB01DC0102C00190B4
:0E1380000D9241505040D8F70895F894FFCFD9
:04138E00FF5A5A00A8
:00000001FF
